:1000000075C099C091C297C096C09AC094C093C061
:1000100092C091C090C08FC039C18DC08CC000000B
:1000200000000000000000000000000023456C9864
:10003000C9FF040714233764A0FFFFFFFFFFFFFF82
:10004000FFFFFFFFFF000000000000000000234052
:100050005F7AB4FFFFFFFFFFFF00140008140008E1
:100060000E140004080E14000305080E1400040802
:100070000A0E1114000305080A0E101400030508E7
:100080000A0E1012140008000E00080E0004080EDC
:10009000000305080E0004080E1100080E1100F3FD
:1000A000F404080E10121400080A0C0E0F1012149B
:1000B00000080EED14000203040500041400040EF1
:1000C0001400040810140004080F1114000305089C
:1000D0000A0E0004080A0E00EEEDECEB140E080404
:1000E0000004080E00EBECEDEEF3F41411241FBE37
:1000F000CFEDCDBF20E0A0E6B0E001C01D92AA3751
:10010000B207E1F7EBE7F0E085E5808781E08383E4
:1001100014821282868311828BE0818788E5828730
:10012000E1E6F0E08DEF87838EEF8583712C552417
:100130005A94ADD021C264CF1BBC19BC18BC089521
:10014000189525B7277E25BF29B7226029BF21E052
:1001500022BF019728F020E188952150E9F7F9CFD7
:10016000089588EE93E0EDCF369A3699FECF95B19B
:100170008091600089270895CF93C72D81E0870D76
:100180008F73782E662D90E0E9D16FEF8C2F90E081
:10019000CF91E4C1FF920F931F93CF93DF93F82E7B
:1001A0000CE710E0CEE7D0E0F11005C0CE01CED1D3
:1001B000F801808304C0F8016081CE01CFD121977E
:1001C0000F5F1F4FC437D10579F7DF91CF911F9192
:1001D0000F91FF900895D0DF81E0DCCF811101C045
:1001E000ABCF815090E0FC01E25EFF4FE491EBBDAC
:1001F000FC01EE5CFF4FE491E9BDFC01EA5BFF4FBF
:10020000849188BD08950F931F93CF93C82F8B01BE
:10021000CC2359F085E0E2DFC80193DF8DDFC80110
:1002200090DFC8018EDFC150F3CFCF911F910F91A6
:100230000895CF93DF93D82F64E170E08AE0E3DF85
:1002400084EF91E07EDF8D2F64E674D1CAE06C2FDD
:1002500071D1892F68EC70E0D6DF83DF8D2F6C2F92
:1002600069D1D92F67D1892F68EC70E0CCDF79DFB5
:1002700068EC70E08D2FC7DF74DF64E170E08AE026
:10028000C2DF84EF91E0DF91CF915BCF18951092A0
:100290007A0087E790E05AD1853519F0612C9BDF11
:1002A00011C0712C872D90E051D1682E8F3F19F02D
:1002B00080E070DF07C0872D91E0970D792E8034A4
:1002C00088F3F6CF90918400D0917E0010917F004A
:1002D000C0917C00CC2319F010E0D0E09AE19F5F40
:1002E00080E040E050E06AE570E0992379F09B01FE
:1002F0002F5F3F4FF9013197E491EE2319F0822FE0
:10030000861BF6CF9150AB01B901EFCF982F6D2F1F
:1003100070E0A82FB0E0E92FF0E0112321F09D015B
:100320002E1B3F0B05C09F0121503109260F371F9F
:100330003197E40FF51F049126593F4FF9010083CF
:10034000915049F78D0F80938600DD2371F01123C2
:1003500029F0282F30E02150310902C020E030E0A0
:10036000F901E659FF4F91E0908397E0980F292F0C
:100370002150E22FE81BF0E0EB51FF4FE491A22F58
:10038000B0E0A659BF4FEC932813F2CFE92FF0E06D
:10039000E759FF4F21E040916A003081431320E08C
:1003A000921B90938700262D253FE8F5352D3D3093
:1003B000B0F4909188009F3F29F480917A00809357
:1003C000880006C091E0960D692E981708F0612C00
:1003D000809188008F5F8F718093880024C0209166
:1003E0007A00209388003132C0F4209181002223CA
:1003F00011F0CC2339F091E0960D692E981798F002
:10040000612C11C0262D6816D9F3662019F02150F1
:10041000622E09C09150692E06C0C111F1CF8091A2
:100420007D00882369F3512C8FEF8DBD80E68CBD54
:10043000AB9A8FE384BB8FE187BB8CEE88BB81E0F6
:1004400083BF91EA9ABD80BF8BB780628BBF8AB7AA
:1004500085608ABF85B7806285BF78948CE287B952
:1004600086EC86B93699FECF8FEF809360008CE2E0
:1004700091E067DE79DEDDDEFACF112416B85CDEAE
:1004800087B38C7E87BBC29820E061E031E040E01A
:1004900050E0E8E0999B06C0CA010197F1F78AB7DE
:1004A00085608ABF86B38E27999B03C0511003C015
:1004B00035C0811107C090E2951590F5211130C02B
:1004C00060E039E0952D71E0923208F070E0970F0E
:1004D000592E913209F4C29A611106C0211103C04C
:1004E000882311F0C29821E0999885B7877E8061B2
:1004F00085BFA895832F887011F480E401C080E641
:10050000816081BD85B7846885BF8B7F85BF789406
:100510008895F89481B58F7B81BDBCCF8111D2CFF6
:100520008FED8DBF1FBEB3DE999A552011F018953F
:1005300001C0A3DF991B79E004C0991F961708F04A
:10054000961B881F7A95C9F780950895E199FECF8B
:100550001FBA8EBBE09A99278DB30895262FE19993
:10056000FECF1CBA1FBA8EBB2DBB0FB6F894E29A11
:0C057000E19A0FBE01960895F894FFCFA9
:00000001FF
